:1000000009C021C020C01FC01EC01DC01CC01BC015
:100010001AC019C011241FBECFE9CDBF10E0A0E661
:10002000B0E0E6EFF3E002C005900D92A036B10714
:10003000D9F710E0A0E6B0E001C01D92A036B107EC
:10004000E1F702D0D6C1DCCF4F925F926F927F92E0
:100050009F92AF92BF92CF92DF92EF92FF920F9357
:100060001F93CF93DF9387E087BB89E088BB82E251
:1000700087B987E886B98FEF9FEF20EF30E0F9016D
:100080003197F1F70197D9F7CC24DD24AA24BB24BA
:1000900066247724992420E040EE442E41E0542E3B
:1000A000369A3699FECF85B1C82FD0E02F96CC0F67
:1000B000DD1FCE018619970997FF03C090958195A2
:1000C0009F4F4F972CF03E01CC24DD24AA24BB2463
:1000D000B39906C0C298CC24DD24AA24BB2447C00F
:1000E0000894A11CB11C84ECA81689E0B80629F478
:1000F0000894C11CD11CAA24BB24CE010F978919D6
:1001000091098C159D0524F4C29A95E0992E02C0A0
:10011000C2989924CE01821B9109C816D9061CF1F8
:10012000B60175956795882777FD8095982F46D0FD
:100130007B018C01B601882777FD8095982F3ED0F2
:1001400020E030E040E05FE398D09B01AC01C801C3
:10015000B7012ED0882339F4C19AC2010197F1F773
:10016000C19825E004C0C2010197F1F720E06E9626
:10017000CC15DD050CF094CF88B38C7F88BB28EEBE
:1001800033E040EF50E005C0CA010197F1F721507C
:10019000304021153105C1F7C29888EE93E0FA018D
:1001A0003197F1F70197D9F7C29A28EE33E0ECCFF7
:1001B00040D008F481E00895E89409C097FB3EF42C
:1001C00090958095709561957F4F8F4F9F4F9923A4
:1001D000A9F0F92F96E9BB279395F6958795779522
:1001E0006795B795F111F8CFFAF4BB0F11F460FFE2
:1001F0001BC06F5F7F4F8F4F9F4F16C0882311F03A
:1002000096E911C0772321F09EE8872F762F05C04D
:10021000662371F096E8862F70E060E02AF09A95E8
:10022000660F771F881FDAF7880F9695879597F9DD
:100230000895990F0008550FAA0BE0E8FEEF161677
:100240001706E807F907C0F012161306E407F507CA
:1002500098F0621B730B840B950B39F40A2661F03E
:10026000232B242B252B21F408950A2609F4A140E1
:10027000A6958FEF811D811D08950AD080C071D091
:1002800028F076D018F0952309F062C067C0ABC0A3
:1002900087D0A8F39923D9F35523C9F3950F50E0DC
:1002A000551FAA27EE27FF27BB2700240894679530
:1002B00020F4E20FF31FB41F0A1E220F331F441F46
:1002C000AA1F6695A9F7779530F4F30FB41F0A1E9D
:1002D000121E08F46395330F441FAA1F221F769540
:1002E00099F7879520F4B40F0A1E121E631F440F5E
:1002F000AA1F221F331F8695A9F7862F712D602D07
:1003000011249F5750408AF0E1F088234AF0EE0F05
:10031000FF1FBB1F661F771F881F91505040A9F712
:100320009E3F510570F014C05EC05F3FECF3983EF5
:10033000DCF3869577956795B795F795E7959F5F79
:10034000C1F7FE2B880F911D9695879597F9089513
:1003500097F99F6780E870E060E008959FEF80EC78
:10036000089500240A94161617061806090608951B
:1003700000240A9412161306140605060895092E81
:100380000394000C11F4882352F0BB0F40F4BF2BF0
:1003900011F460FF04C06F5F7F4F8F4F9F4F089530
:1003A00057FD9058440F551F59F05F3F71F0479526
:1003B000880F97FB991F61F09F3F79F0879508950B
:1003C000121613061406551FF2CF4695F1DF08C02A
:1003D000161617061806991FF1CF86957105610547
:1003E00008940895E894BB2766277727CB0197F9EF
:0603F0000895F894FFCF10
:00000001FF
